:020000040000FA
:040000008A013C280D
:0A000600F039860005150511080009
:1000100085100B288514A0000320200E032001303A
:1000200012200800A200F930A1000000A10B152841
:10003000A20B13280800A5002930A502A503250856
:100040002920A600A608031928280A20A50A1F2887
:1000500008008207503452344534533445344E340A
:1000600054344534003420345434413452344A3406
:100070004534543441340034831603132030850052
:100080000F3086009B0107309C009D0183120313F3
:1000900085018601831603131930990004309800F6
:1000A00083120313903098009813103012203030D0
:1000B000042005301220303004200530122030306A
:1000C0000420053012202030042005301220283072
:1000D0000B200C300B2001300B2006300B202A3077
:1000E0001B20C030082033301B207B281812181624
:1000F0001A081A081A080D30A300981701301220A8
:100100008C1E80281A08A40023088207B628B3286A
:10011000B028AD28AA28A728A428A1289E289B2873
:10012000982895282408A700B8282408A800B828EB
:100130002408A900B8282408AA00B8282408AB007D
:10014000B8282408AC00B8282408AD00B828240832
:10015000AE00B8282408AF00B8282408B000B8289A
:100160002408B100B8282408B200B8282408B30035
:10017000A30B802898130130122001300820013091
:10018000122020300A2020300A2027080A202808C0
:100190000A2029080A202A080A202B080A202C08ED
:1001A0000A20C0300820013012202D080A202E0815
:1001B0000A202F080A2030080A2031080A203208B5
:0401C0000A20762873
:00000001FF
